:020000040010EA
:100000000F0000EAFEFFFFEAFEFFFFEAFEFFFFEA45
:10001000FEFFFFEAFEFFFFEA260000EA0090A0E1F3
:10002000040198E5D3F021E30E502DE90FE0A0E1A3
:1000300010FF2FE10E50BDE8D1F021E30900A0E14F
:1000400004F05EE2C8D09FE5C8009FE50FE0A0E1A4
:1000500010FF2FE10D00A0E1D1F021E3B8809FE572
:10006000D2F021E300D0A0E1600040E213F021E3F0
:1000700000D0A0E1A4109FE5A4209FE5A4309FE557
:10008000030052E10400913404008234FBFFFF3A84
:100090000000A0E390109FE590209FE5020051E151
:1000A00004008134FCFFFF3A84E09FE584009FE573
:1000B00010FF2FE1FEFFFFEA04E04EE200402DE9D1
:1000C00000E04FE100402DE901002DE948E09FE507
:1000D00000019EE500E18EE513F021E30E502DE9CD
:1000E0000FE0A0E110FF2FE10E50BDE892F021E3F8
:1000F00024E09FE530E18EE50100BDE80040BDE869
:100100000EF06FE10080FDE8FEFFFFEAFEFFFFEA70
:10011000FEFFFFEA004020000D05100000F0FFFF89
:10012000080810000000200008002000080020003F
:1001300008002000B40010003902100000B581B0A2
:1001400000230093074B0F21584300F0A5FA02E06B
:10015000009B01330093009B8342F9D301B001BCA3
:1001600000470000B6BB0000F0B5030C1E0681B0CE
:10017000320E00920127730F720003D43B4205D068
:10018000312050E03B424DD132204CE0040A300F88
:100190003840303000F07EF9F00E3840303000F05A
:1001A00079F9B00E3840303000F074F9700E3840F4
:1001B000303000F06FF9009838402406303000F0FD
:1001C00069F9E00F303000F065F9A00F38403030A9
:1001D00000F060F9600F3840303000F05BF9200F1C
:1001E0003840303000F056F9E00E38403030250EFF
:1001F00000F050F9A00E640E38403C4030303034EE
:100200003D4000F047F93035201C00F043F9281C30
:1002100000F040F92C2000F03DF90D2000F03AF9F3
:100220000A2003E0332000F035F92C2000F032F9E9
:1002300001B0F0BC01BC0047F0B5264B44221A6166
:10024000254A264B81B09A6000F010F9244800F04E
:100250003FF900F0A7F9234800F03AF9224A802339
:100260009B02136013618023DB0213601361802300
:100270001B031360136180235B03136013611A4D2A
:1002800080239B028027802680242B633F037603F4
:10029000E40201200093FFF751FF2F6301202E633A
:1002A0002C63FFF74BFF6C630120FFF747FFAA2188
:1002B0000E4800F0C7F9041C0120FFF73FFF009B28
:1002C000201C6B636F636E63FFF74EFF0120FFF727
:1002D00035FFD4E700FCFFFF010000A500FDFFFF94
:1002E000F0071000FC07100000F4FFFFAAAA0000AE
:1002F00010B50006040E0A2C02D10D2000F0CAF839
:10030000201C00F0C7F810BC01BC00470FB4F0B5CA
:1003100086B00BAB20CB059304E0002800D1A0E011
:10032000FFF7E6FF287801352528F6D12878013532
:10033000302804D0202802D00022019209E02A7837
:10034000131C303B1B061F0E0135092F03D90190EA
:10035000101C002703E02B7801900135181C6C2835
:1003600001D04C2801D12878013558283FD0582891
:100370000DD849282ED0492804D8432817D044281E
:10038000CED127E0532817D05528C9D120E06928BD
:1003900020D0692804D8632809D06428C0D119E086
:1003A000752815D0782822D07328B9D104E0059A91
:1003B0001078131D0593B3E7059A1468131D059370
:1003C00002E0FFF795FF013420780028F9D1A9E772
:1003D0000A220DE0059A131D05931468002C03DA18
:1003E0002D206442FFF784FF0A23009305E01022CA
:1003F0000598031D009205930468002202AB6E4627
:10040000DA721336201C009900F08CF930300006A7
:10041000000E392802D9C31D1B06180E013E30708C
:100420000099201C00F038F9041C002F02D07B1E1C
:100430001B061F0E002CE5D1391C321C03E06B4655
:100440001B79013E33707B1E1B061F0EFF2FF6D15A
:10045000541A02E0FFF74CFF013420780028F9D14C
:1004600060E706B0F0BC08BC04B01847074B602238
:100470001A60074B1A68AC2313608C231B0153606E
:100480001A231362502313607047000004F4FFFF27
:1004900000002000034B1A6853699907FCD5D0610E
:1004A000D0697047000020000A2807D1074B1A685E
:1004B00053699907FCD50D23D361D369034B1A689F
:1004C00053699907FCD5D061D069704700002000BE
:1004D00010B5041C02E00134FFF7E6FF2078002885
:1004E000F9D110BC02BC0847024B1B6858690123B4
:1004F0001840704700002000034B1A685369D90761
:10050000FCD5906970470000000020001A4A802343
:100510005B001366194A80231B025360184A194B6B
:100520001A62184A936ED907FBD5174BD362154B45
:100530009B6E5A07FBD5134A936E1907FBD504230C
:10054000136310498B6E1A07FBD50B6B0322134301
:100550000B630C4B9B6E1907FBD50C4A0C4B0D49DA
:10056000DA670D4A0123013304C11F2BFBD10B4A6B
:100570000B4B9A637047000000FFFFFF40FDFFFF39
:100580000106000000FCFFFF0E1C480008011000DF
:1005900004F0FFFF84F0FFFF0C01100010011000B9
:1005A000FCF0FFFF0D4B20221A610D4BE022D2011F
:1005B0001A606C3B1A6060331A600A4A80231B0180
:1005C000136753601361084B1A688123136001237A
:1005D000136011235360054B1363704700FCFFFF4A
:1005E00070F4FFFF00F4FFFF0400200003FF00FF92
:1005F000084B1A68136B00061363000E1369990504
:10060000FCD5D0601369D907FCD590680006000EB0
:100610007047000004002000094B19680B6B802212
:10062000134300040B63000C0B699A05FCD5C860EA
:100630000B69DA07FCD588680004000C70470000DD
:1006400004002000F0B5124E32680D06136B1149FC
:100650000B401363136B08273B4300041363000C28
:10066000FFF7DAFF3168FF230A6B1B061A430A63A0
:100670000B6B2D0EBB430B63041C281CFFF7B8FF4C
:100680002402044B04431C40201CF0BC02BC08475D
:1006900004002000FFFFFF00002934D001230022C6
:1006A00010B488422CD301242407A14204D28142F1
:1006B00002D209011B01F8E7E400A14204D2814201
:1006C00002D249005B00F8E7884201D3401A1A437E
:1006D0004C08A04202D3001B5C0822438C08A042B5
:1006E00002D3001B9C082243CC08A04202D3001B6B
:1006F000DC082243002803D01B0901D00909E3E7E5
:10070000101C10BC704702B500F070F8002006BC49
:100710001047000003B5FFF7BFFF0EBC4243891A24
:100720001847C04600295AD00123884200D270479A
:1007300010B401242407A14204D2814202D209014B
:100740001B01F8E7E400A14204D2814202D2490031
:100750005B00F8E70022884200D3401A4C08A04210
:1007600005D3001B9C460124E3411A4363468C08D1
:10077000A04205D3001B9C460224E3411A43634672
:10078000CC08A04205D3001B9C460324E3411A4336
:1007900063469C46002803D01B0901D00909D9E70C
:1007A0000E242407224018D063460724234214D085
:1007B00063460324E3411A4201D0CC080019634682
:1007C0000224E3411A4201D08C0800196346012437
:1007D000E3411A4201D04C08001910BC704702B521
:1007E00000F004F8002006BC1047C0467047C04621
:1007F0005541525420494E49540D0A005350492046
:08080000494E49540D0A0000A5
:080808000000FCFF0000FEFFF0
:0400000500100000E7
:00000001FF
